:020000040000FA
:10020000AEEF01F09EA8FED70950AD6E1200ABA272
:1002100002D0AB98AB889EAAFED7AE50096E1200F2
:1002200089688A6A8B68F00E926E3F0E936E9F0EFD
:10023000946EC60EC16EC00EC26E400EAF6EFB0E47
:10024000AC14AC6E200EAC10AC6E100EAB10AB6EDE
:10025000800EAB10AB6E016A81B0FED7F00E036E5C
:10026000800E046E1A0E056E060E066E076A0750A3
:10027000000808E10650000805E10550000802E109
:100280000450000807BED8804AE2010E045C096EE3
:10029000000E0A6ED8A00A3C055E000E0A6ED8A0B9
:1002A0000A3C065E000E0A6ED8A00A3C075E0950A2
:1002B000046E000E075C08E1040E065C05E1930E77
:1002C000055C02E1E00E045C02E307AE03D0010E20
:1002D0000310036E000E075C08E1030E065C05E1E7
:1002E0000D0E055C02E1400E045C02E307AE03D094
:1002F000020E0310036E000E075C08E1010E065C9F
:1003000005E1860E055C02E1A00E045C02E307AE87
:1003100003D0040E0310036E0350896EA8D78968BA
:10032000026807EC01F00950026E086A02A203D0CD
:1003300002A001D0082A085202E1770E016E02B431
:1003400002D0F70E016E02B602D07F0E016E02508F
:10035000896E0150096E02EC01F0E2D710EF01F056
:020000040030CA
:0E000000FFFEF6FEFFFEFBFFF03FFF9FFFBF7F
:00000001FF
